:1000000093C00000ACC00000AAC00000A8C000005F
:10001000A6C00000A4C00000A2C00000A0C0000054
:100020009EC000009CC000009AC0000029C60000CD
:1000300096C0000094C0000092C0000090C0000074
:100040008EC000008CC000008AC00000DFC000002D
:1000500086C0000084C0000082C0000026C20000EC
:100060007EC000000CC100007AC0000078C0000013
:1000700076C000001201100102000008EB034B20C3
:1000800000000102030109024300020100C032091D
:1000900004000001020201000524001001052401F2
:1000A0000301042402060524060001070582030853
:1000B000000209040100020A000000070504021002
:1000C000000007058302100000040309042803440C
:1000D000006F006E0061006C006400200044006549
:1000E000006C006D00610072002000440061007629
:1000F000006900730000003003420065006E006973
:100100000074006F003700670000001A03300030F1
:10011000003000300030003000300030003000305F
:10012000003000320000000011241FBECFEFD2E0EB
:10013000DEBFCDBF11E0A0E0B1E0E4E1FEE002C02F
:1001400005900D92AC31B107D9F712E0ACE1B1E006
:1001500001C01D92A633B107E1F765D159C650CF52
:100160004FB7F8942091310230913202FC01318373
:1001700020834FBF089580911D01882331F080E2D4
:1001800091E0EEDF10921D0108958CE390E060E2B3
:1001900071E0CBD2882339F080E291E0E1DF8BEB94
:1001A00090E060E0E5C2089580911E01882331F05F
:1001B00082E291E0D5DF10921E0108958CE390E079
:1001C00062E271E0B2D2882339F082E291E0C8DFC6
:1001D00084ED90E060E0CCC2089580911F018823F7
:1001E00031F084E291E0BCDF10921F01089582E0BB
:1001F00090E064E271E099D2882339F084E291E0E2
:10020000AFDF8DEE90E060E0B3C208951F920F92D1
:100210000FB60F9211248F939F938091310290918A
:100220003202019690933202809331029F918F9116
:100230000F900FBE0F901F90189587E296E061E037
:1002400097C284E892E060E093D287E296E060E0B3
:100250008FC282E068E070E041EC20E00ED383E0E2
:1002600060E170E041E824E008D384E060E170E000
:1002700040E824E002D384E892E061E079C21F9272
:100280000F920FB60F9211242F933F934F935F93CA
:100290006F937F938F939F93AF93BF93EF93FF934E
:1002A00080912F02882331F08BEA91E01BD280935A
:1002B000CE0002C010921C01FF91EF91BF91AF914F
:1002C0009F918F917F916F915F914F913F912F916E
:1002D0000F900FBE0F901F901895809119018130DB
:1002E00021F0823021F080E003C080E301C080E291
:1002F00090911801923009F4886090911A0196301B
:1003000011F4826007C0973011F4846003C0983004
:1003100009F4866092E09093C80098ED9093C9002C
:100320008093CA00209114013091150140E050E003
:1003300060E472E48FE090E049D521503040309382
:10034000CD002093CC000895E4E1F1E09091F1001C
:100350004091F100813239F0823209F448C0803294
:1003600009F060C022C0613A09F05CC08091E800E9
:10037000877F8093E80081918093F10081E0EB31E9
:10038000F807C9F78091E8008E7F8093E80080919C
:10039000E80080FFFCCF8091E80082FFFCCF8091D5
:1003A000E8008B7F8093E80008956132D9F5809151
:1003B000E800877F8093E8008091E80082FFFCCF0F
:1003C0008091F100819381E0EB31F807C9F78091CA
:1003D000E8008B7F8093E80080DF8091E8008E7FCB
:1003E0008093E8008091E80080FD1CC0FBCF613263
:1003F000C9F4342F20E0892F90E0822B932B80FFCB
:1004000003C081E080931F018091E800877F809383
:10041000E8008091E8008E7F8093E8008091E800FA
:1004200080FFFCCF08951F93CF93DF9384B7877F1E
:1004300084BF88E10FB6F89480936000109260004A
:100440000FBE90E080E80FB6F8948093610090931F
:1004500061000FBE8DE787BD82E084BD93E095BD4E
:1004600080936E003ADF8BEA91E0F5D086E291E06E
:10047000F2D015E010933002F5D110933002C0E0B5
:10048000D1E08A81882319F0E881F98109952496C1
:1004900081E0C431D807A9F76497F3CF81E0809356
:1004A0001E0184ED90E061E063C11F920F920FB6D0
:1004B0000F9211242F933F934F935F936F937F93EA
:1004C0008F939F93AF93BF93EF93FF936091CE0071
:1004D00086E291E0D2D0E2DFFF91EF91BF91AF9140
:1004E0009F918F917F916F915F914F913F912F914C
:1004F0000F900FBE0F901F90189581E080931D0103
:100500008BEB90E061E034C11F938091350288232A
:1005100009F45AC084E08093E9008091E80085FDE9
:100520000BC013C080912F028038E1F36091F1007D
:100530008BEA91E0A2D0E1DF8091F200882391F76D
:100540008091E8008F778093E80080912F028823C4
:1005500081F080911C01882361F481E080931C016B
:100560008BEA91E0BFD09091C80095FFFCCF8093BB
:10057000CE0083E08093E9008091AA01882321F1D5
:100580008091E80085FFFCCF1091F20005C086E263
:1005900091E0A8D08093F1008091AA01882321F0F6
:1005A0008091F200803198F38091E8008F778093FA
:1005B000E800103149F48091E80085FFFCCF80917C
:1005C000E8008F778093E8001F910895692F7727BF
:1005D0006230710539F06330710549F061307105A1
:1005E000B1F521C083E490E0E6E8F0E025C090702A
:1005F0008130910569F08130910538F082309105A4
:1006000051F083309105A1F40BC0E9ECF0E005C096
:10061000EDECF0E002C0E7EFF0E0849190E00CC078
:10062000EBE0F1E0FACF82E190E0E4E7F0E004C033
:1006300080E090E0E0E0F0E0309759F0DA011196C8
:10064000FC93EE93F9019183808381E0089580E02B
:10065000089580E008952FB7F894FC01E058FF4F0B
:1006600091838083FC01EE57FF4F918380838C57E9
:100670009F4FFC0110822FBF08957FB7F894FC01B3
:10068000EC57FF4F20812038A1F4FC01EE57FF4FBB
:10069000208131812F5F3F4F318320834081518101
:1006A0009C0120583F4F4217530731F491838083B8
:1006B00003C020812F5F2083FC01E058FF4FA08101
:1006C000B1816C93208131812F5F3F4F3183208333
:1006D000A081B181AE17BF0719F411969C938E9338
:1006E0007FBF08951F939C011FB7F894FC01EE573C
:1006F000FF4FA081B1818C91408151814F5F5F4F4D
:1007000051834083D901AC57BF4F9C9191509C932A
:1007100060817181A90140585F4F6417750711F41A
:10072000318320831FBF1F910895FB014FB7F894B9
:1007300020913102309132024FBF40815181241704
:10074000350738F0B901641B750B6817790760F03D
:1007500007C040955095420F531F4817590730F076
:100760003183208381E0089580E0089580E008953A
:10077000E0E0F1E008C0208131812817390711F449
:100780006283089534962091300230E0220F331FA7
:10079000220F331F20503F4FE217F30761F70895F0
:1007A00080913502882309F04CDD64D266D2109224
:1007B000350210923402109233028091D8008F7764
:1007C0008093D80019BC0895DF93CF9300D000D058
:1007D000CDB7DEB74FD251D210923502109233020C
:1007E00019BC89B5826089BD09B400FEFDCF809136
:1007F000D800982F9F779093D80080688093D80076
:10080000809163008E7F809363008091D8008F7DFC
:100810008093D80080E091E060E0AE014F5F5F4FD1
:100820009E012D5F3F4FD2DE882331F0E981FA81AE
:100830003796E491E0931B018091E0008E7F8093D6
:10084000E0008091E20081608093E2008091E2000C
:1008500088608093E2000F900F900F900F90CF91DF
:10086000DF91089580913402882309F099DF81E0B7
:1008700080933402A9DF789408958093E9008091F1
:10088000EB0081608093EB004093EC008091ED00E1
:100890008270282B77706930710540F061317105E5
:1008A00038F06132710530F480E205C080E003C0A9
:1008B00080E101C080E3822B8093ED008091ED0008
:1008C00082608093ED000895E1EFF0E0208130E058
:1008D0004081942F80E0282B392BC9010895EF9295
:1008E000FF920F931F93DF93CF93CDB7DEB7299776
:1008F0000FB6F894DEBF0FBECDBF6091F1007091CE
:10090000F100753009F4C1C0763048F4713009F453
:100910006DC0713070F0733009F07CC167C0783001
:1009200009F432C1793009F44AC1763009F072C154
:10093000CCC0062F10E0C801807E9070009709F0AF
:1009400069C10F7110700330110509F463C1809102
:10095000F1008091F100B8DF0130110599F102300A
:10096000110531F10115110509F056C180913302CD
:1009700090E0926060E0AE014F5F5F4F9E01295FA3
:100980003F4F24DE882309F447C1E981FA81379675
:10099000E491F0E0CF01807C9070009711F082E04C
:1009A00001C080E0E07AF070309769F081600BC0A0
:1009B0008093E9009091EB0081E090FD80E010923F
:1009C000E90001C080E09091E800977F9093E800F3
:1009D0008093F1001092F1008091E8008E7F809367
:1009E000E8008091E80082FFFCCFE3C0062F10E012
:1009F0009801207E30702115310509F00BC10F716F
:100A000010700330110509F405C179875DDF7C01A1
:100A10005BDFAC0179850230110509F0FDC0E114FE
:100A2000F10409F0F9C08093E9008091EB0080FFA8
:100A300029C041155105D9F07130A1F48091EB0026
:100A400080618093EB0021E030E002C0220F331F71
:100A50004A95E2F72093EA001092EA008091EB00B9
:100A6000886003C08091EB0080628093EB0010925D
:100A7000E9008091E800877F8093E8008091E8009A
:100A80008E7F9AC01092E900C7C0662309F0C2C0E9
:100A90008091F1009091E3008F739078892B80937F
:100AA000E3008091E800877F8093E8008091E80070
:100AB0008E7F8093E8008091E80080FFFCCF8091DA
:100AC000E30080688093E300A7C0FEDE8C01FCDEBB
:100AD0008987FADEF82EE92EC8016985AE014D5FDF
:100AE0005F4F9E01295F3F4F71DD882309F494C059
:100AF0008091E800877F8093E8002F813885A701E7
:100B0000852F942F2817390708F4C90160911B011C
:100B10009C011DC04091E80040FD0EC0FBCFEB8161
:100B2000FC81AF014F5F5F4F5C834B83E491E093A7
:100B3000F1002150304031F05091F20040911B0102
:100B4000541768F34091E8004E7F4093E800211568
:100B5000310521F04091E80042FFDCCF2091E80010
:100B600022FD27C070E01ED1009749F48091E80073
:100B700080FFFCCF8091E8008E7F8093E800809119
:100B8000E80082FFFCCF15C0603809F043C08091B7
:100B9000E800877F8093E800809133028093F10022
:100BA0008091E8008E7F8093E8008091E80082FFCA
:100BB000FCCF8091E8008B7F8093E8002DC06623F6
:100BC00049F582DE8C01E090330280E091E060E044
:100BD000AE014B5F5F4F9E01295F3F4FF7DC8823DB
:100BE000D9F0ED81FE817196E491F0E0E017F10714
:100BF00098F08091E800877F8093E80000933302AB
:100C00008091E8008E7F8093E800EE2009F4C9D03F
:100C100020DB02C0872F98DB8091E80083FF0AC0A9
:100C20008091EB0080628093EB008091E800877FE9
:100C30008093E80029960FB6F894DEBF0FBECDBFB3
:100C4000CF91DF911F910F91FF90EF9008951F9327
:100C500080913502882361F01091E900177010929D
:100C6000E9008091E80083FF01C039DE1093E900BC
:100C70001F9108951092E20008951092E1000895E6
:100C80001F920F920FB60F9211242F933F934F9301
:100C90005F936F937F938F939F93AF93BF93EF93E4
:100CA000FF938091E10080FF1DC08091E20080FFF2
:100CB00019C08091E1008E7F8093E1008091E20075
:100CC0008E7F8093E2008091E20080618093E20059
:100CD0008091D80080628093D80019BC62D01092B5
:100CE0003502AFDA8091E10084FF24C08091E200F8
:100CF00084FF20C019BC89B5826089BD09B400FE9B
:100D0000FDCF8091D8008F7D8093D8008091E10045
:100D10008F7E8093E1008091E2008F7E8093E200DD
:100D20008091E20081608093E20081E0809335024F
:100D300084DA37D08091E10083FF22C08091E20005
:100D400083FF1EC08091E100877F8093E1001092B5
:100D500033028091E1008E7F8093E1008091E20078
:100D60008E7F8093E2008091E20080618093E200B8
:100D700060911B0180E070E040E020E07EDD11D05A
:100D8000FF91EF91BF91AF919F918F917F916F9163
:100D90005F914F913F912F910F900FBE0F901F9039
:100DA00018950895AA1BBB1B51E107C0AA1FBB1FC2
:100DB000A617B70710F0A61BB70B881F991F5A95E7
:100DC000A9F780959095BC01CD010895A1E21A2E56
:100DD000AA1BBB1BFD010DC0AA1FBB1FEE1FFF1FDF
:100DE000A217B307E407F50720F0A21BB30BE40B2F
:100DF000F50B661F771F881F991F1A9469F7609576
:100E00007095809590959B01AC01BD01CF0108952F
:040E1000F894FFCF84
:100E14002706000084020000ED000000D40000005A
:0C0E2400BB000000004B000000000808AC
:00000001FF
